
mips16-elf.x:     file format elf32-bigmips


Disassembly of section .text:

00fe1400 <null>:
  fe1400:	e820      	jr	ra
  fe1402:	6500      	nop

00fe1404 <return_zero>:
  fe1404:	e820      	jr	ra
  fe1406:	6a00      	li	v0,0

00fe1408 <return_one>:
  fe1408:	e820      	jr	ra
  fe140a:	6a01      	li	v0,1

00fe140c <return_intsize>:
  fe140c:	e820      	jr	ra
  fe140e:	6a04      	li	v0,4

00fe1410 <return_pointersize>:
  fe1410:	e820      	jr	ra
  fe1412:	6a04      	li	v0,4

00fe1414 <return_short>:
  fe1414:	6a12      	li	v0,18
  fe1416:	e820      	jr	ra
  fe1418:	ea4b      	neg	v0
  fe141a:	6500      	nop

00fe141c <return_long>:
  fe141c:	b202      	lw	v0,fe1424 <return_long+0x8>
  fe141e:	e820      	jr	ra
  fe1420:	6500      	nop
  fe1422:	6500      	nop
  fe1424:	ffee      	daddiu	a3,sp,56
  fe1426:	ddcc      	sw	a2,48(a1)

00fe1428 <return_arg1>:
  fe1428:	e820      	jr	ra
  fe142a:	6744      	move	v0,a0

00fe142c <return_arg2>:
  fe142c:	e820      	jr	ra
  fe142e:	6745      	move	v0,a1

00fe1430 <inc>:
  fe1430:	e820      	jr	ra
  fe1432:	4441      	addiu	v0,a0,1

00fe1434 <add>:
  fe1434:	e820      	jr	ra
  fe1436:	e4a9      	addu	v0,a0,a1

00fe1438 <add3>:
  fe1438:	e4a9      	addu	v0,a0,a1
  fe143a:	e820      	jr	ra
  fe143c:	e2c9      	addu	v0,a2
  fe143e:	6500      	nop

00fe1440 <load>:
  fe1440:	e820      	jr	ra
  fe1442:	9c40      	lw	v0,0(a0)

00fe1444 <store>:
  fe1444:	6aff      	li	v0,255
  fe1446:	e820      	jr	ra
  fe1448:	dc40      	sw	v0,0(a0)
  fe144a:	6500      	nop

00fe144c <load_long>:
  fe144c:	e820      	jr	ra
  fe144e:	9c40      	lw	v0,0(a0)

00fe1450 <store_long>:
  fe1450:	b202      	lw	v0,fe1458 <store_long+0x8>
  fe1452:	e820      	jr	ra
  fe1454:	dc40      	sw	v0,0(a0)
  fe1456:	6500      	nop
  fe1458:	fedc      	dla	a2,fe14c8 <call_complex+0x4>
  fe145a:	ba98      	lwu	a0,96(v0)

00fe145c <member>:
  fe145c:	6a01      	li	v0,1
  fe145e:	dc41      	sw	v0,4(a0)
  fe1460:	e820      	jr	ra
  fe1462:	9c42      	lw	v0,8(a0)

00fe1464 <get_global>:
  fe1464:	675c      	move	v0,gp
  fe1466:	f2e0 9a44 	lw	v0,740(v0)
  fe146a:	e820      	jr	ra
  fe146c:	6500      	nop
  fe146e:	6500      	nop

00fe1470 <set_global>:
  fe1470:	675c      	move	v0,gp
  fe1472:	f2e0 da84 	sw	a0,740(v0)
  fe1476:	e820      	jr	ra
  fe1478:	6500      	nop
  fe147a:	6500      	nop

00fe147c <set_stack>:
  fe147c:	63ff      	addiu	sp,-8
  fe147e:	6afe      	li	v0,254
  fe1480:	d200      	sw	v0,0(sp)
  fe1482:	6aff      	li	v0,255
  fe1484:	d201      	sw	v0,4(sp)
  fe1486:	e820      	jr	ra
  fe1488:	6301      	addiu	sp,8
  fe148a:	6500      	nop

00fe148c <use_stack>:
  fe148c:	63ff      	addiu	sp,-8
  fe148e:	6afe      	li	v0,254
  fe1490:	d200      	sw	v0,0(sp)
  fe1492:	6aff      	li	v0,255
  fe1494:	d201      	sw	v0,4(sp)
  fe1496:	9300      	lw	v1,0(sp)
  fe1498:	9201      	lw	v0,4(sp)
  fe149a:	e349      	addu	v0,v1,v0
  fe149c:	e820      	jr	ra
  fe149e:	6301      	addiu	sp,8

00fe14a0 <call_null>:
  fe14a0:	63fd      	addiu	sp,-24
  fe14a2:	6204      	sw	ra,16(sp)
  fe14a4:	1be1 8528 	jal	fe14a0 <call_null>
  fe14a8:	6500      	nop
  fe14aa:	9704      	lw	a3,16(sp)
  fe14ac:	ef00      	jr	a3
  fe14ae:	6303      	addiu	sp,24

00fe14b0 <call_simple>:
  fe14b0:	63fd      	addiu	sp,-24
  fe14b2:	6204      	sw	ra,16(sp)
  fe14b4:	1be1 850a 	jal	fe1428 <return_arg1>
  fe14b8:	6cfe      	li	a0,254
  fe14ba:	4a01      	addiu	v0,1
  fe14bc:	9704      	lw	a3,16(sp)
  fe14be:	ef00      	jr	a3
  fe14c0:	6303      	addiu	sp,24
  fe14c2:	6500      	nop

00fe14c4 <call_complex>:
  fe14c4:	63fd      	addiu	sp,-24
  fe14c6:	6205      	sw	ra,20(sp)
  fe14c8:	d004      	sw	s0,16(sp)
  fe14ca:	6705      	move	s0,a1
  fe14cc:	1be1 850a 	jal	fe1428 <return_arg1>
  fe14d0:	6785      	move	a0,a1
  fe14d2:	677c      	move	v1,gp
  fe14d4:	f2e0 db44 	sw	v0,740(v1)
  fe14d8:	6750      	move	v0,s0
  fe14da:	9705      	lw	a3,20(sp)
  fe14dc:	9004      	lw	s0,16(sp)
  fe14de:	ef00      	jr	a3
  fe14e0:	6303      	addiu	sp,24
  fe14e2:	6500      	nop

00fe14e4 <call_pointer>:
  fe14e4:	63fd      	addiu	sp,-24
  fe14e6:	6204      	sw	ra,16(sp)
  fe14e8:	f6df 6a10 	li	v0,65232
  fe14ec:	ea40      	jalr	v0
  fe14ee:	6500      	nop
  fe14f0:	9704      	lw	a3,16(sp)
  fe14f2:	ef00      	jr	a3
  fe14f4:	6303      	addiu	sp,24
  fe14f6:	6500      	nop

00fe14f8 <condition>:
  fe14f8:	2402      	beqz	a0,fe14fe <condition+0x6>
  fe14fa:	6a0a      	li	v0,10
  fe14fc:	dc40      	sw	v0,0(a0)
  fe14fe:	e820      	jr	ra
  fe1500:	6a00      	li	v0,0
  fe1502:	6500      	nop

00fe1504 <loop>:
  fe1504:	6a00      	li	v0,0
  fe1506:	6762      	move	v1,v0
  fe1508:	ea82      	slt	v0,a0
  fe150a:	6004      	bteqz	fe1514 <loop+0x10>
  fe150c:	e269      	addu	v0,v1
  fe150e:	4b01      	addiu	v1,1
  fe1510:	eb82      	slt	v1,a0
  fe1512:	61fc      	btnez	fe150c <loop+0x8>
  fe1514:	e820      	jr	ra
  fe1516:	6500      	nop

00fe1518 <main>:
  fe1518:	e820      	jr	ra
  fe151a:	6a00      	li	v0,0
